:020000000528D1
:08000800D628831600308600A3
:100010000F30850081128312051620308400800184
:10002000840A041F0F28AA0AF0308600C420860E16
:10003000C4208601CF200314860DCF20031C1C286A
:10004000860193202308A8000310230D82070000D7
:1000500021280030742801307428003069280230CB
:100060007428000021280130692800005B28033033
:10007000742800004C2800002128000021280230AC
:100080006928000021280000602800004728F0307F
:100090008600A220A400702896308600A220A0002E
:1000A000C4202A1C7128A1018601A901AA1C2128AB
:1000B0000130A800742878308600A220AA00702899
:1000C000E13086009320031023080F3C0319052814
:1000D0007028A100013021183330A118703086003B
:1000E000C420290886002128A200210803197C28A1
:1000F0002808A80E2118A8042808A90086000310C3
:10010000200820072007A500A50D250DA700210820
:10011000A500A50D250D2207A7072408C038AE208D
:100120002708AE202128A30105080F39031D9428B4
:1001300005080F390319982805080F390319080015
:10014000A3049C2805080F390319A228A5008600DE
:100150000310A50C2508251903300800A500BE20B2
:100160000930A60005120314BE20A50C0318BA28F6
:100170000512BB280516A60BB42808000B1DBE28C7
:10018000E63081000B1108000608CF208601CF2041
:100190008600CF208601CF208600CF200800A60150
:0E01A000A501A50FD128A60BD1280800090043
:02400E00F13F80
:00000001FF
